:0200000480007A
:100000009717000093870701B7000000B7110000A1
:10001000B7F2FFFFB7FEFF7FB70F008023A01700E6
:1000200023A2370023A4570023A6D70123A8F70152
:1000300097170000938707FD171800001308C8FEE4
:1000400003A1070003A2070003A3070003AE0700F4
:1000500003AF07003701008037F2FF7F370300004E
:10006000371E000037FFFFFF23202800232248000F
:10007000232468002326C8012328E80197180000DC
:100080009388C8FBB77072429380F0E6B75734127A
:100090009387876737EFBC9A130F0FEF3771724260
:1000A0001301F1E63758341213088867B7EFBC9A8A
:1000B000938F0FEF23A0180023A2F80023A4E801D8
:1000C00023A6280023A8080123AAF8011715000079
:1000D000130545F4971500009385C5F7370610F012
:1000E0001306C6F26306B5028326C5002320D60098
:1000F000832685002320D600832645002320D600B2
:10010000832605002320D600130505016FF09FFD0F
:10011000370510F0130505F223200500000000004C
:0401200000000000DB
:10100000111111110000000000000000000000009C
:10101000FFFFFFFFFFFFFFFFFFFFFFFFFFFFFFFFE0
:10102000FFFFFFFFFFFFFFFFFFFFFFFFFFFFFFFFD0
:10103000FFFFFFFFFFFFFFFFFFFFFFFFFFFFFFFFC0
:10104000FFFFFFFFFFFFFFFFFFFFFFFFFFFFFFFFB0
:040000058000000077
:00000001FF
